:1000000000308A0004280000FF238316900000308F
:100010008A003F288316851283128516000000008F
:100020008316851283128512000000342830840064
:100030008313000803192A280130A100A001A00B96
:100040001F28A10B1E284A30A000A00B2528282815
:10005000800B1C2800341230A802031C3E282830D4
:1000600084008313FC3080050310800C800C000892
:1000700003193E283C280000800B3B2800348401F3
:1000800083131F3083051F1383161F109F101F112A
:100090009F110730831299001F1383161F109F10A2
:1000A0001F119F1183121F1083160108C7390838CA
:1000B00081008312900107309900831605080330F0
:1000C0008312A000A00B622819088C1183169901D5
:1000D0008312A601A5012608233C031C7A28031DD0
:1000E00075282508273C031C7A280A20A50A03192D
:1000F000A60A6B281C30A8001620A601A501A60898
:10010000031D8B282508193C031C8B280A20A50AEF
:100110000319A60A7F280130A80016200330A70083
:100120007A30A8002B20A70B9028A601A501A608CD
:10013000031DA3282508163C031CA3280A20A50A92
:100140000319A60A97280330A80016200230A7003A
:10015000AC30A8002B20A70BA828A601A501A60853
:10016000031DBB282508193C031CBB280A20A50A2F
:100170000319A60AAF283F30A8001620A601A50142
:10018000A608031DCC282508593C031CCC280A20AE
:10019000A50A0319A60AC0281C30A8001620A6012B
:1001A000A501A608031DDD282508193C031CDD2830
:1001B0000A20A50A0319A60AD1280130A800162092
:1001C0000330A7007A30A8002B20A70BE228A60155
:1001D000A501A608031DF5282508163C031CF528D3
:1001E0000A20A50A0319A60AE9280330A800162048
:1001F0000230A700AC30A8002B20A70BFA28A601DC
:10020000A501A608031D0D292508193C031C0D296D
:100210000A20A50A0319A60A01290430A700FA300A
:0C022000A8001620A70B0F296928630016
:02400E00F5318A
:00000001FF
